BL51 BANKED LINKER/LOCATER V6.05                                                        08/18/2015  10:55:48  PAGE 1


BL51 BANKED LINKER/LOCATER V6.05, INVOKED BY:
C:\KEIL\C51\BIN\BL51.EXE 1602-wendu.obj TO 1602-wendu


MEMORY MODEL: SMALL WITH FLOATING POINT ARITHMETIC


INPUT MODULES INCLUDED:
  1602-wendu.obj (1602_WENDU)
  C:\KEIL\C51\LIB\C51FPS.LIB (?C?FPADD)
  C:\KEIL\C51\LIB\C51FPS.LIB (?C?FPMUL)
  C:\KEIL\C51\LIB\C51FPS.LIB (?C?FCAST)
  C:\KEIL\C51\LIB\C51FPS.LIB (?C?CASTF)
  C:\KEIL\C51\LIB\C51FPS.LIB (?C?FPGETOPN)
  C:\KEIL\C51\LIB\C51S.LIB (?C_STARTUP)
  C:\KEIL\C51\LIB\C51S.LIB (?C?COPY)
  C:\KEIL\C51\LIB\C51S.LIB (?C?CLDOPTR)
  C:\KEIL\C51\LIB\C51S.LIB (?C?UIDIV)
  C:\KEIL\C51\LIB\C51S.LIB (?C?LNEG)
  C:\KEIL\C51\LIB\C51S.LIB (ABS)


LINK MAP OF MODULE:  1602-wendu (1602_WENDU)


            TYPE    BASE      LENGTH    RELOCATION   SEGMENT NAME
            -----------------------------------------------------

            * * * * * * *   D A T A   M E M O R Y   * * * * * * *
            REG     0000H     0008H     ABSOLUTE     "REG BANK 0"
                    0008H     0018H                  *** GAP ***
            BIT     0020H.0   0000H.1   UNIT         _BIT_GROUP_
                    0020H.1   0000H.7                *** GAP ***
            DATA    0021H     001DH     UNIT         _DATA_GROUP_
            IDATA   003EH     0001H     UNIT         ?STACK

            * * * * * * *   C O D E   M E M O R Y   * * * * * * *
            CODE    0000H     0003H     ABSOLUTE     
            CODE    0003H     0443H     UNIT         ?C?LIB_CODE
            CODE    0446H     00C9H     UNIT         ?PR?_DISPLAY?1602_WENDU
            CODE    050FH     0061H     UNIT         ?PR?GETTMPVALUE?1602_WENDU
            CODE    0570H     0057H     UNIT         ?PR?_WRITEBYTE?1602_WENDU
            CODE    05C7H     0040H     UNIT         ?PR?MAIN?1602_WENDU
            CODE    0607H     002AH     UNIT         ?PR?_WRITESTRING?1602_WENDU
            CODE    0631H     0024H     UNIT         ?PR?READBIT?1602_WENDU
            CODE    0655H     0024H     UNIT         ?PR?READBYTE?1602_WENDU
            CODE    0679H     001FH     UNIT         ?PR?DSINIT?1602_WENDU
            CODE    0698H     001EH     UNIT         ?PR?_DELAYMS?1602_WENDU
            CODE    06B6H     001CH     UNIT         ?CO?1602_WENDU
            CODE    06D2H     001AH     UNIT         ?PR?INIT?1602_WENDU
            CODE    06ECH     0016H     UNIT         ?PR?DSWAIT?1602_WENDU
            CODE    0702H     0012H     UNIT         ?PR?_WRITECOMM?1602_WENDU
            CODE    0714H     0012H     UNIT         ?PR?_WRITEDATA?1602_WENDU
            CODE    0726H     000CH     UNIT         ?C_C51STARTUP
            CODE    0732H     000CH     UNIT         ?PR?_ABS?ABS
            CODE    073EH     0008H     UNIT         ?PR?SENDCHANGECMD?1602_WENDU
            CODE    0746H     0008H     UNIT         ?PR?SENDREADCMD?1602_WENDU
            CODE    074EH     0002H     UNIT         ?PR?DELAYUS?1602_WENDU
BL51 BANKED LINKER/LOCATER V6.05                                                      08/18/2015  10:55:48  PAGE 2





OVERLAY MAP OF MODULE:   1602-wendu (1602_WENDU)


SEGMENT                                 BIT_GROUP          DATA_GROUP 
  +--> CALLED SEGMENT                START    LENGTH     START    LENGTH
------------------------------------------------------------------------
?C_C51STARTUP                        -----    -----      -----    -----
  +--> ?PR?MAIN?1602_WENDU

?PR?MAIN?1602_WENDU                  -----    -----      0021H    0011H
  +--> ?CO?1602_WENDU
  +--> ?PR?SENDCHANGECMD?1602_WENDU
  +--> ?PR?INIT?1602_WENDU
  +--> ?PR?_WRITECOMM?1602_WENDU
  +--> ?PR?_WRITESTRING?1602_WENDU
  +--> ?PR?_DELAYMS?1602_WENDU
  +--> ?PR?GETTMPVALUE?1602_WENDU
  +--> ?PR?_DISPLAY?1602_WENDU

?PR?SENDCHANGECMD?1602_WENDU         -----    -----      -----    -----
  +--> ?PR?_WRITEBYTE?1602_WENDU

?PR?_WRITEBYTE?1602_WENDU            0020H.0  0000H.1    -----    -----
  +--> ?PR?DSINIT?1602_WENDU
  +--> ?PR?DSWAIT?1602_WENDU
  +--> ?PR?_DELAYMS?1602_WENDU

?PR?INIT?1602_WENDU                  -----    -----      -----    -----
  +--> ?PR?_WRITECOMM?1602_WENDU

?PR?_WRITECOMM?1602_WENDU            -----    -----      -----    -----
  +--> ?PR?DELAYUS?1602_WENDU
  +--> ?PR?_DELAYMS?1602_WENDU

?PR?_WRITESTRING?1602_WENDU          -----    -----      0039H    0005H
  +--> ?PR?_WRITEDATA?1602_WENDU

?PR?_WRITEDATA?1602_WENDU            -----    -----      -----    -----
  +--> ?PR?DELAYUS?1602_WENDU
  +--> ?PR?_DELAYMS?1602_WENDU

?PR?GETTMPVALUE?1602_WENDU           -----    -----      0032H    0006H
  +--> ?PR?SENDREADCMD?1602_WENDU
  +--> ?PR?READBYTE?1602_WENDU

?PR?SENDREADCMD?1602_WENDU           -----    -----      -----    -----
  +--> ?PR?_WRITEBYTE?1602_WENDU

?PR?READBYTE?1602_WENDU              -----    -----      -----    -----
  +--> ?PR?READBIT?1602_WENDU

?PR?READBIT?1602_WENDU               0020H.0  0000H.1    -----    -----

?PR?_DISPLAY?1602_WENDU              -----    -----      0032H    0007H
BL51 BANKED LINKER/LOCATER V6.05                                                      08/18/2015  10:55:48  PAGE 3


  +--> ?CO?1602_WENDU
  +--> ?PR?_ABS?ABS
  +--> ?PR?_WRITECOMM?1602_WENDU
  +--> ?PR?_WRITESTRING?1602_WENDU
  +--> ?PR?_WRITEDATA?1602_WENDU



SYMBOL TABLE OF MODULE:  1602-wendu (1602_WENDU)

  VALUE           TYPE          NAME
  ----------------------------------

  -------         MODULE        1602_WENDU
  C:0000H         SYMBOL        _ICE_DUMMY_
  D:0080H         PUBLIC        P0
  D:0090H         PUBLIC        P1
  D:00A0H         PUBLIC        P2
  D:00B0H         PUBLIC        P3
  C:073EH         PUBLIC        sendChangeCmd
  D:00A8H         PUBLIC        IE
  D:00B8H         PUBLIC        IP
  B:00B0H.5       PUBLIC        RS
  C:05C7H         PUBLIC        main
  B:00A0H.6       PUBLIC        dula
  C:0607H         PUBLIC        _writeString
  C:0714H         PUBLIC        _writeData
  B:00A0H.7       PUBLIC        wela
  D:0098H         PUBLIC        SCON
  C:0655H         PUBLIC        readByte
  D:0088H         PUBLIC        TCON
  C:06D2H         PUBLIC        init
  C:0702H         PUBLIC        _writeComm
  C:0631H         PUBLIC        readBit
  C:0746H         PUBLIC        sendReadCmd
  C:06BCH         SYMBOL        _?ix1000
  C:06C1H         SYMBOL        _?ix1001
  C:057FH         PUBLIC        _writeByte
  C:0698H         PUBLIC        _delayMs
  B:00A0H.2       PUBLIC        ds
  C:074EH         PUBLIC        delayUs
  B:00B0H.4       PUBLIC        LCDEN
  D:00C8H         PUBLIC        T2CON
  B:00B0H.6       PUBLIC        rw
  C:0679H         PUBLIC        dsInit
  C:06ECH         PUBLIC        dsWait
  C:050FH         PUBLIC        getTmpValue
  C:0446H         PUBLIC        _display
  D:00D0H         PUBLIC        PSW
  -------         PROC          DELAYUS
  C:074EH         LINE#         28
  C:074EH         LINE#         29
  C:074EH         LINE#         30
  C:074FH         LINE#         31
  -------         ENDPROC       DELAYUS
  -------         PROC          _DELAYMS
  D:0006H         SYMBOL        a
BL51 BANKED LINKER/LOCATER V6.05                                                      08/18/2015  10:55:48  PAGE 4


  -------         DO            
  D:0006H         SYMBOL        i
  D:0004H         SYMBOL        j
  -------         ENDDO         
  C:0698H         LINE#         33
  C:0698H         LINE#         34
  C:0698H         LINE#         36
  C:06A1H         LINE#         37
  C:06B5H         LINE#         38
  -------         ENDPROC       _DELAYMS
  -------         PROC          _WRITECOMM
  D:0007H         SYMBOL        comm
  C:0702H         LINE#         41
  C:0702H         LINE#         42
  C:0702H         LINE#         43
  C:0704H         LINE#         44
  C:0706H         LINE#         45
  C:0708H         LINE#         46
  C:070BH         LINE#         47
  C:070DH         LINE#         48
  -------         ENDPROC       _WRITECOMM
  -------         PROC          _WRITEDATA
  D:0007H         SYMBOL        dat
  C:0714H         LINE#         52
  C:0714H         LINE#         53
  C:0714H         LINE#         54
  C:0716H         LINE#         55
  C:0718H         LINE#         56
  C:071AH         LINE#         57
  C:071DH         LINE#         58
  C:071FH         LINE#         59
  -------         ENDPROC       _WRITEDATA
  -------         PROC          INIT
  C:06D2H         LINE#         63
  C:06D2H         LINE#         64
  C:06D2H         LINE#         65
  C:06D4H         LINE#         66
  C:06D8H         LINE#         67
  C:06DDH         LINE#         68
  C:06E2H         LINE#         69
  C:06E7H         LINE#         70
  -------         ENDPROC       INIT
  -------         PROC          _WRITESTRING
  D:0039H         SYMBOL        str
  D:003CH         SYMBOL        length
  -------         DO            
  D:003DH         SYMBOL        i
  -------         ENDDO         
  C:0607H         LINE#         73
  C:060FH         LINE#         74
  C:060FH         LINE#         76
  C:0619H         LINE#         77
  C:0619H         LINE#         78
  C:062CH         LINE#         79
  C:0630H         LINE#         80
  -------         ENDPROC       _WRITESTRING
  -------         PROC          DSINIT
BL51 BANKED LINKER/LOCATER V6.05                                                      08/18/2015  10:55:48  PAGE 5


  -------         DO            
  D:0006H         SYMBOL        i
  -------         ENDDO         
  C:0679H         LINE#         84
  C:0679H         LINE#         85
  C:0679H         LINE#         88
  C:067BH         LINE#         89
  C:067FH         LINE#         90
  C:0688H         LINE#         91
  C:068AH         LINE#         92
  C:068EH         LINE#         93
  C:0697H         LINE#         94
  -------         ENDPROC       DSINIT
  -------         PROC          DSWAIT
  -------         DO            
  D:0006H         SYMBOL        i
  -------         ENDDO         
  C:06ECH         LINE#         96
  C:06ECH         LINE#         97
  C:06ECH         LINE#         99
  C:06EFH         LINE#         100
  C:06F4H         LINE#         101
  C:06F8H         LINE#         102
  C:0701H         LINE#         103
  -------         ENDPROC       DSWAIT
  -------         PROC          READBIT
  -------         DO            
  D:0006H         SYMBOL        i
  B:0020H.0       SYMBOL        b
  -------         ENDDO         
  C:0631H         LINE#         106
  C:0631H         LINE#         107
  C:0631H         LINE#         110
  C:0633H         LINE#         111
  C:0637H         LINE#         112
  C:0639H         LINE#         113
  C:0641H         LINE#         114
  C:0645H         LINE#         115
  C:0649H         LINE#         116
  C:0652H         LINE#         117
  C:0654H         LINE#         118
  -------         ENDPROC       READBIT
  -------         PROC          READBYTE
  -------         DO            
  D:0002H         SYMBOL        i
  D:0007H         SYMBOL        j
  D:0005H         SYMBOL        dat
  -------         ENDDO         
  C:0655H         LINE#         120
  C:0655H         LINE#         121
  C:0655H         LINE#         124
  C:0657H         LINE#         125
  C:0659H         LINE#         126
  C:0659H         LINE#         127
  C:065FH         LINE#         129
  C:066BH         LINE#         130
  C:0676H         LINE#         131
BL51 BANKED LINKER/LOCATER V6.05                                                      08/18/2015  10:55:48  PAGE 6


  C:0678H         LINE#         132
  -------         ENDPROC       READBYTE
  -------         PROC          L?0078
  -------         ENDPROC       L?0078
  -------         PROC          _WRITEBYTE
  D:0007H         SYMBOL        dat
  -------         DO            
  D:0002H         SYMBOL        i
  D:0006H         SYMBOL        j
  B:0020H.0       SYMBOL        b
  -------         ENDDO         
  C:057FH         LINE#         135
  C:057FH         LINE#         136
  C:057FH         LINE#         140
  C:0581H         LINE#         141
  C:0581H         LINE#         142
  C:0585H         LINE#         143
  C:0589H         LINE#         145
  C:058CH         LINE#         146
  C:058CH         LINE#         147
  C:0596H         LINE#         148
  C:0598H         LINE#         149
  C:05A7H         LINE#         150
  C:05A7H         LINE#         152
  C:05A7H         LINE#         153
  C:05A9H         LINE#         154
  C:05B6H         LINE#         155
  C:05B8H         LINE#         156
  C:05C2H         LINE#         157
  C:05C2H         LINE#         158
  C:05C6H         LINE#         159
  -------         ENDPROC       _WRITEBYTE
  -------         PROC          SENDCHANGECMD
  C:073EH         LINE#         162
  C:073EH         LINE#         163
  C:073EH         LINE#         164
  C:073EH         LINE#         165
  C:073EH         LINE#         166
  C:073EH         LINE#         167
  C:0741H         LINE#         168
  -------         ENDPROC       SENDCHANGECMD
  -------         PROC          SENDREADCMD
  C:0746H         LINE#         171
  C:0746H         LINE#         172
  C:0746H         LINE#         173
  C:0746H         LINE#         174
  C:0746H         LINE#         175
  C:0746H         LINE#         176
  C:0749H         LINE#         177
  -------         ENDPROC       SENDREADCMD
  -------         PROC          GETTMPVALUE
  -------         DO            
  D:0006H         SYMBOL        tmpvalue
  D:0032H         SYMBOL        value
  D:0034H         SYMBOL        t
  D:0001H         SYMBOL        low
  D:0007H         SYMBOL        high
BL51 BANKED LINKER/LOCATER V6.05                                                      08/18/2015  10:55:48  PAGE 7


  -------         ENDDO         
  C:050FH         LINE#         181
  C:050FH         LINE#         182
  C:050FH         LINE#         187
  C:0512H         LINE#         189
  C:0517H         LINE#         190
  C:051AH         LINE#         192
  C:051AH         LINE#         193
  C:051CH         LINE#         194
  C:051EH         LINE#         195
  C:0522H         LINE#         197
  C:053CH         LINE#         199
  C:056FH         LINE#         201
  C:056FH         LINE#         202
  -------         ENDPROC       GETTMPVALUE
  -------         PROC          _DISPLAY
  D:0032H         SYMBOL        v
  -------         DO            
  D:0003H         SYMBOL        count
  D:0034H         SYMBOL        datas
  D:0002H         SYMBOL        tmp
  -------         ENDDO         
  C:0446H         LINE#         204
  C:044AH         LINE#         205
  C:044AH         LINE#         207
  C:045DH         LINE#         208
  C:0468H         LINE#         209
  C:0471H         LINE#         210
  C:048BH         LINE#         211
  C:04A5H         LINE#         212
  C:04BFH         LINE#         213
  C:04CCH         LINE#         214
  C:04D1H         LINE#         215
  C:04DCH         LINE#         216
  C:04DCH         LINE#         217
  C:04E0H         LINE#         218
  C:04E2H         LINE#         220
  C:04E2H         LINE#         221
  C:04EBH         LINE#         222
  C:04EBH         LINE#         223
  C:04EFH         LINE#         224
  C:04EFH         LINE#         225
  C:04F5H         LINE#         226
  C:04F5H         LINE#         227
  C:04F7H         LINE#         228
  C:04F7H         LINE#         229
  C:0502H         LINE#         230
  C:0505H         LINE#         231
  C:0505H         LINE#         232
  C:050AH         LINE#         233
  C:050AH         LINE#         234
  C:050EH         LINE#         235
  -------         ENDPROC       _DISPLAY
  -------         PROC          MAIN
  -------         DO            
  D:0021H         SYMBOL        table
  -------         ENDDO         
BL51 BANKED LINKER/LOCATER V6.05                                                      08/18/2015  10:55:48  PAGE 8


  C:05C7H         LINE#         238
  C:05C7H         LINE#         239
  C:05C7H         LINE#         240
  C:05DAH         LINE#         241
  C:05DDH         LINE#         242
  C:05E0H         LINE#         243
  C:05E5H         LINE#         244
  C:05F0H         LINE#         245
  C:05F0H         LINE#         246
  C:05F0H         LINE#         247
  C:05F7H         LINE#         248
  C:05FCH         LINE#         249
  C:0602H         LINE#         250
  C:0605H         LINE#         251
  -------         ENDPROC       MAIN
  -------         ENDMOD        1602_WENDU

  -------         MODULE        ?C?FPADD
  C:000AH         PUBLIC        ?C?FPADD
  C:0006H         PUBLIC        ?C?FPSUB
  -------         ENDMOD        ?C?FPADD

  -------         MODULE        ?C?FPMUL
  C:00FBH         PUBLIC        ?C?FPMUL
  -------         ENDMOD        ?C?FPMUL

  -------         MODULE        ?C?FCAST
  C:020BH         PUBLIC        ?C?FCASTC
  C:0206H         PUBLIC        ?C?FCASTI
  C:0201H         PUBLIC        ?C?FCASTL
  -------         ENDMOD        ?C?FCAST

  -------         MODULE        ?C?CASTF
  C:023FH         PUBLIC        ?C?CASTF
  -------         ENDMOD        ?C?CASTF

  -------         MODULE        ?C?COPY
  C:0390H         PUBLIC        ?C?COPY
  -------         ENDMOD        ?C?COPY

  -------         MODULE        ?C?CLDOPTR
  C:03B6H         PUBLIC        ?C?CLDOPTR
  -------         ENDMOD        ?C?CLDOPTR

  -------         MODULE        ?C?UIDIV
  C:03E3H         PUBLIC        ?C?UIDIV
  -------         ENDMOD        ?C?UIDIV

  -------         MODULE        ?C?LNEG
  C:0438H         PUBLIC        ?C?LNEG
  -------         ENDMOD        ?C?LNEG

  -------         MODULE        ABS
  C:0732H         PUBLIC        _ABS
  -------         ENDMOD        ABS

Program Size: data=38.1 xdata=0 code=1872
BL51 BANKED LINKER/LOCATER V6.05                                                      08/18/2015  10:55:48  PAGE 9


LINK/LOCATE RUN COMPLETE.  0 WARNING(S),  0 ERROR(S)
